 javaw

 Timestamp is ffffffff (Sun Feb  7 06:28:15 2106)

 Preferred load address is 00400000

 Start         Length     Name                   Class
 0001:00000000 00000d49H .text$mn                CODE
 0002:00000000 000000ecH .idata$5                DATA
 0002:000000ec 00000004H .00cfg                  DATA
 0002:000000f0 00000004H .CRT$XCA                DATA
 0002:000000f4 00000004H .CRT$XCAA               DATA
 0002:000000f8 00000004H .CRT$XCZ                DATA
 0002:000000fc 00000004H .CRT$XIA                DATA
 0002:00000100 00000004H .CRT$XIAA               DATA
 0002:00000104 00000004H .CRT$XIAC               DATA
 0002:00000108 00000004H .CRT$XIZ                DATA
 0002:0000010c 00000004H .CRT$XPA                DATA
 0002:00000110 00000004H .CRT$XPZ                DATA
 0002:00000114 00000004H .CRT$XTA                DATA
 0002:00000118 00000008H .CRT$XTZ                DATA
 0002:0000011c 00000000H .gfids$y                DATA
 0002:00000120 00000190H .rdata                  DATA
 0002:000002b0 00000004H .rdata$sxdata           DATA
 0002:000002b4 000002b0H .rdata$zzzdbg           DATA
 0002:00000564 00000004H .rtc$IAA                DATA
 0002:00000568 00000004H .rtc$IZZ                DATA
 0002:0000056c 00000004H .rtc$TAA                DATA
 0002:00000570 00000008H .rtc$TZZ                DATA
 0002:00000578 0000003cH .xdata$x                DATA
 0002:000005b4 00000000H .edata                  DATA
 0002:000005b4 000000b4H .idata$2                DATA
 0002:00000668 00000014H .idata$3                DATA
 0002:0000067c 000000ecH .idata$4                DATA
 0002:00000768 000004dcH .idata$6                DATA
 0003:00000000 00000030H .data                   DATA
 0003:00000030 0000037cH .bss                    DATA
 0004:00000000 00000270H .rsrc$01                DATA
 0004:00000270 00006578H .rsrc$02                DATA

  Address         Publics by Value              Rva+Base       Lib:Object

 0000:00000000       ___guard_fids_table        00000000     <absolute>
 0000:00000000       ___enclave_config          00000000     <absolute>
 0000:00000000       ___hybrid_code_map         00000000     <absolute>
 0000:00000000       ___hybrid_code_map_count   00000000     <absolute>
 0000:00000000       ___guard_iat_table         00000000     <absolute>
 0000:00000000       ___volatile_metadata       00000000     <absolute>
 0000:00000000       ___guard_longjmp_table     00000000     <absolute>
 0000:00000000       ___guard_iat_count         00000000     <absolute>
 0000:00000000       ___dynamic_value_reloc_table 00000000     <absolute>
 0000:00000000       ___guard_longjmp_count     00000000     <absolute>
 0000:00000000       ___hybrid_auxiliary_iat    00000000     <absolute>
 0000:00000000       ___guard_fids_count        00000000     <absolute>
 0000:00000001       ___safe_se_handler_count   00000001     <absolute>
 0000:00000100       ___guard_flags             00000100     <absolute>
 0000:00000000       ___ImageBase               00400000     <linker-defined>
 0001:00000000       _WinMain@16                00401000 f   main.obj
 0001:000000db       ___local_stdio_printf_options 004010db f i main.obj
 0001:000000e1       __vfprintf_l               004010e1 f i main.obj
 0001:00000105       _printf                    00401105 f i main.obj
 0001:00000123       _JLI_MemAlloc@4            00401123 f   jli:jli.dll
 0001:00000129       _JLI_GetStdArgs@0          00401129 f   jli:jli.dll
 0001:0000012f       _JLI_GetStdArgc@0          0040112f f   jli:jli.dll
 0001:00000135       _JLI_CmdToArgs@4           00401135 f   jli:jli.dll
 0001:0000013b       _JLI_InitArgProcessing@8   0040113b f   jli:jli.dll
 0001:00000141       _JLI_Launch@56             00401141 f   jli:jli.dll
 0001:00000388       _WinMainCRTStartup         00401388 f   MSVCRT:exe_winmain.obj
 0001:000003d6       ___scrt_acquire_startup_lock 004013d6 f   MSVCRT:utility.obj
 0001:00000408       ___scrt_initialize_crt     00401408 f   MSVCRT:utility.obj
 0001:00000441       ___scrt_initialize_onexit_tables 00401441 f   MSVCRT:utility.obj
 0001:000004e6       ___scrt_is_nonwritable_in_current_image 004014e6 f   MSVCRT:utility.obj
 0001:0000057a       ___scrt_release_startup_lock 0040157a f   MSVCRT:utility.obj
 0001:00000597       ___scrt_uninitialize_crt   00401597 f   MSVCRT:utility.obj
 0001:000005bf       __onexit                   004015bf f   MSVCRT:utility.obj
 0001:000005fa       _atexit                    004015fa f   MSVCRT:utility.obj
 0001:0000065c       ___security_init_cookie    0040165c f   MSVCRT:gs_support.obj
 0001:000006a7       __get_startup_new_mode     004016a7 f   MSVCRT:new_mode.obj
 0001:000006a7       ___scrt_exe_initialize_mta 004016a7 f   MSVCRT:utility_desktop.obj
 0001:000006a7       __get_startup_commit_mode  004016a7 f   MSVCRT:commit_mode.obj
 0001:000006a7       __matherr                  004016a7 f   MSVCRT:matherr.obj
 0001:000006a7       __get_startup_thread_locale_mode 004016a7 f   MSVCRT:thread_locale.obj
 0001:000006a7       ___scrt_initialize_winrt   004016a7 f   MSVCRT:utility_desktop.obj
 0001:000006a7       ___scrt_stub_for_initialize_mta 004016a7 f   MSVCRT:utility_desktop.obj
 0001:000006aa       __get_startup_argv_mode    004016aa f   MSVCRT:argv_mode.obj
 0001:000006ae       __get_startup_file_mode    004016ae f   MSVCRT:file_mode.obj
 0001:000006b4       ?__scrt_initialize_type_info@@YAXXZ 004016b4 f   MSVCRT:tncleanup.obj
 0001:000006c0       ___scrt_stub_for_acrt_initialize 004016c0 f   MSVCRT:ucrt_stubs.obj
 0001:000006c0       ___scrt_stub_for_acrt_uninitialize 004016c0 f   MSVCRT:ucrt_stubs.obj
 0001:000006c0       ___vcrt_uninitialize       004016c0 f   MSVCRT:ucrt_stubs.obj
 0001:000006c0       __should_initialize_environment 004016c0 f   MSVCRT:env_mode.obj
 0001:000006c0       ___acrt_uninitialize       004016c0 f   MSVCRT:ucrt_stubs.obj
 0001:000006c0       ___vcrt_initialize         004016c0 f   MSVCRT:ucrt_stubs.obj
 0001:000006c0       ___acrt_initialize         004016c0 f   MSVCRT:ucrt_stubs.obj
 0001:000006c3       __initialize_default_precision 004016c3 f   MSVCRT:default_precision.obj
 0001:000006e4       @_guard_check_icall_nop@4  004016e4 f   MSVCRT:guard_support.obj
 0001:000006e4       __initialize_denormal_control 004016e4 f   MSVCRT:denormal_control.obj
 0001:000006e4       __initialize_invalid_parameter_handler 004016e4 f   MSVCRT:invalid_parameter_handler.obj
 0001:000006e5       ___local_stdio_scanf_options 004016e5 f i MSVCRT:default_local_stdio_options.obj
 0001:000006eb       ___scrt_initialize_default_local_stdio_options 004016eb f   MSVCRT:default_local_stdio_options.obj
 0001:00000708       ___scrt_is_user_matherr_present 00401708 f   MSVCRT:matherr_detection.obj
 0001:00000714       ___scrt_get_dyn_tls_init_callback 00401714 f   MSVCRT:dyn_tls_init.obj
 0001:0000071a       ___scrt_get_dyn_tls_dtor_callback 0040171a f   MSVCRT:dyn_tls_dtor.obj
 0001:00000720       ___scrt_fastfail           00401720 f   MSVCRT:utility_desktop.obj
 0001:0000083a       ___scrt_get_show_window_mode 0040183a f   MSVCRT:utility_desktop.obj
 0001:0000086b       ___scrt_initialize_mta     0040186b f   MSVCRT:utility_desktop.obj
 0001:00000870       ___scrt_is_managed_app     00401870 f   MSVCRT:utility_desktop.obj
 0001:000008b3       ___scrt_set_unhandled_exception_filter 004018b3 f   MSVCRT:utility_desktop.obj
 0001:000008bf       ___scrt_unhandled_exception_filter@4 004018bf f   MSVCRT:utility_desktop.obj
 0001:00000900       __crt_debugger_hook        00401900 f   MSVCRT:utility_desktop.obj
 0001:00000908       __RTC_Initialize           00401908 f   MSVCRT:initsect.obj
 0001:00000934       __RTC_Terminate            00401934 f   MSVCRT:initsect.obj
 0001:00000960       __SEH_prolog4              00401960 f   MSVCRT:sehprolg4.obj
 0001:000009a6       __SEH_epilog4              004019a6 f   MSVCRT:sehprolg4.obj
 0001:000009bb       __except_handler4          004019bb f   MSVCRT:chandler4gs.obj
 0001:000009de       ___isa_available_init      004019de f   MSVCRT:cpu_disp.obj
 0001:00000b75       ___scrt_is_ucrt_dll_in_use 00401b75 f   MSVCRT:ucrt_detection.obj
 0001:00000b81       @__security_check_cookie@4 00401b81 f   MSVCRT:secchk.obj
 0001:00000b92       ___raise_securityfailure   00401b92 f   MSVCRT:gs_report.obj
 0001:00000bba       ___report_gsfailure        00401bba f   MSVCRT:gs_report.obj
 0001:00000cb3       _IsProcessorFeaturePresent@4 00401cb3 f   kernel32:KERNEL32.dll
 0001:00000cb9       _memset                    00401cb9 f   vcruntime:VCRUNTIME140.dll
 0001:00000cbf       __except_handler4_common   00401cbf f   vcruntime:VCRUNTIME140.dll
 0001:00000cc5       __seh_filter_exe           00401cc5 f   ucrt:api-ms-win-crt-runtime-l1-1-0.dll
 0001:00000ccb       __set_app_type             00401ccb f   ucrt:api-ms-win-crt-runtime-l1-1-0.dll
 0001:00000cd1       ___setusermatherr          00401cd1 f   ucrt:api-ms-win-crt-math-l1-1-0.dll
 0001:00000cd7       __configure_narrow_argv    00401cd7 f   ucrt:api-ms-win-crt-runtime-l1-1-0.dll
 0001:00000cdd       __initialize_narrow_environment 00401cdd f   ucrt:api-ms-win-crt-runtime-l1-1-0.dll
 0001:00000ce3       __get_narrow_winmain_command_line 00401ce3 f   ucrt:api-ms-win-crt-runtime-l1-1-0.dll
 0001:00000ce9       __initterm                 00401ce9 f   ucrt:api-ms-win-crt-runtime-l1-1-0.dll
 0001:00000cef       __initterm_e               00401cef f   ucrt:api-ms-win-crt-runtime-l1-1-0.dll
 0001:00000cf5       _exit                      00401cf5 f   ucrt:api-ms-win-crt-runtime-l1-1-0.dll
 0001:00000cfb       __exit                     00401cfb f   ucrt:api-ms-win-crt-runtime-l1-1-0.dll
 0001:00000d01       __set_fmode                00401d01 f   ucrt:api-ms-win-crt-stdio-l1-1-0.dll
 0001:00000d07       __cexit                    00401d07 f   ucrt:api-ms-win-crt-runtime-l1-1-0.dll
 0001:00000d0d       __c_exit                   00401d0d f   ucrt:api-ms-win-crt-runtime-l1-1-0.dll
 0001:00000d13       __register_thread_local_exe_atexit_callback 00401d13 f   ucrt:api-ms-win-crt-runtime-l1-1-0.dll
 0001:00000d19       __configthreadlocale       00401d19 f   ucrt:api-ms-win-crt-locale-l1-1-0.dll
 0001:00000d1f       __set_new_mode             00401d1f f   ucrt:api-ms-win-crt-heap-l1-1-0.dll
 0001:00000d25       ___p__commode              00401d25 f   ucrt:api-ms-win-crt-stdio-l1-1-0.dll
 0001:00000d2b       __initialize_onexit_table  00401d2b f   ucrt:api-ms-win-crt-runtime-l1-1-0.dll
 0001:00000d31       __register_onexit_function 00401d31 f   ucrt:api-ms-win-crt-runtime-l1-1-0.dll
 0001:00000d37       __crt_atexit               00401d37 f   ucrt:api-ms-win-crt-runtime-l1-1-0.dll
 0001:00000d3d       __controlfp_s              00401d3d f   ucrt:api-ms-win-crt-runtime-l1-1-0.dll
 0001:00000d43       _terminate                 00401d43 f   ucrt:api-ms-win-crt-runtime-l1-1-0.dll
 0002:00000000       __imp__InitializeSListHead@4 00402000     kernel32:KERNEL32.dll
 0002:00000004       __imp__GetStartupInfoW@4   00402004     kernel32:KERNEL32.dll
 0002:00000008       __imp__SetUnhandledExceptionFilter@4 00402008     kernel32:KERNEL32.dll
 0002:0000000c       __imp__TerminateProcess@8  0040200c     kernel32:KERNEL32.dll
 0002:00000010       __imp__GetCurrentProcess@0 00402010     kernel32:KERNEL32.dll
 0002:00000014       __imp__GetModuleHandleW@4  00402014     kernel32:KERNEL32.dll
 0002:00000018       __imp__UnhandledExceptionFilter@4 00402018     kernel32:KERNEL32.dll
 0002:0000001c       __imp__GetCommandLineA@0   0040201c     kernel32:KERNEL32.dll
 0002:00000020       __imp__QueryPerformanceCounter@4 00402020     kernel32:KERNEL32.dll
 0002:00000024       __imp__GetCurrentProcessId@0 00402024     kernel32:KERNEL32.dll
 0002:00000028       __imp__GetCurrentThreadId@0 00402028     kernel32:KERNEL32.dll
 0002:0000002c       __imp__GetSystemTimeAsFileTime@4 0040202c     kernel32:KERNEL32.dll
 0002:00000030       __imp__IsDebuggerPresent@0 00402030     kernel32:KERNEL32.dll
 0002:00000034       __imp__IsProcessorFeaturePresent@4 00402034     kernel32:KERNEL32.dll
 0002:00000038       \177KERNEL32_NULL_THUNK_DATA 00402038     kernel32:KERNEL32.dll
 0002:0000003c       __imp___except_handler4_common 0040203c     vcruntime:VCRUNTIME140.dll
 0002:00000040       __imp__memset              00402040     vcruntime:VCRUNTIME140.dll
 0002:00000044       \177VCRUNTIME140_NULL_THUNK_DATA 00402044     vcruntime:VCRUNTIME140.dll
 0002:00000048       __imp__getenv              00402048     ucrt:api-ms-win-crt-environment-l1-1-0.dll
 0002:0000004c       __imp____p__environ        0040204c     ucrt:api-ms-win-crt-environment-l1-1-0.dll
 0002:00000050       \177api-ms-win-crt-environment-l1-1-0_NULL_THUNK_DATA 00402050     ucrt:api-ms-win-crt-environment-l1-1-0.dll
 0002:00000054       __imp___set_new_mode       00402054     ucrt:api-ms-win-crt-heap-l1-1-0.dll
 0002:00000058       \177api-ms-win-crt-heap-l1-1-0_NULL_THUNK_DATA 00402058     ucrt:api-ms-win-crt-heap-l1-1-0.dll
 0002:0000005c       __imp___configthreadlocale 0040205c     ucrt:api-ms-win-crt-locale-l1-1-0.dll
 0002:00000060       \177api-ms-win-crt-locale-l1-1-0_NULL_THUNK_DATA 00402060     ucrt:api-ms-win-crt-locale-l1-1-0.dll
 0002:00000064       __imp____setusermatherr    00402064     ucrt:api-ms-win-crt-math-l1-1-0.dll
 0002:00000068       \177api-ms-win-crt-math-l1-1-0_NULL_THUNK_DATA 00402068     ucrt:api-ms-win-crt-math-l1-1-0.dll
 0002:0000006c       __imp____p___argv          0040206c     ucrt:api-ms-win-crt-runtime-l1-1-0.dll
 0002:00000070       __imp___controlfp_s        00402070     ucrt:api-ms-win-crt-runtime-l1-1-0.dll
 0002:00000074       __imp___crt_atexit         00402074     ucrt:api-ms-win-crt-runtime-l1-1-0.dll
 0002:00000078       __imp___seh_filter_exe     00402078     ucrt:api-ms-win-crt-runtime-l1-1-0.dll
 0002:0000007c       __imp___set_app_type       0040207c     ucrt:api-ms-win-crt-runtime-l1-1-0.dll
 0002:00000080       __imp____p___argc          00402080     ucrt:api-ms-win-crt-runtime-l1-1-0.dll
 0002:00000084       __imp__terminate           00402084     ucrt:api-ms-win-crt-runtime-l1-1-0.dll
 0002:00000088       __imp___initialize_narrow_environment 00402088     ucrt:api-ms-win-crt-runtime-l1-1-0.dll
 0002:0000008c       __imp___get_narrow_winmain_command_line 0040208c     ucrt:api-ms-win-crt-runtime-l1-1-0.dll
 0002:00000090       __imp___initterm           00402090     ucrt:api-ms-win-crt-runtime-l1-1-0.dll
 0002:00000094       __imp___initterm_e         00402094     ucrt:api-ms-win-crt-runtime-l1-1-0.dll
 0002:00000098       __imp__exit                00402098     ucrt:api-ms-win-crt-runtime-l1-1-0.dll
 0002:0000009c       __imp___exit               0040209c     ucrt:api-ms-win-crt-runtime-l1-1-0.dll
 0002:000000a0       __imp___cexit              004020a0     ucrt:api-ms-win-crt-runtime-l1-1-0.dll
 0002:000000a4       __imp___c_exit             004020a4     ucrt:api-ms-win-crt-runtime-l1-1-0.dll
 0002:000000a8       __imp___register_thread_local_exe_atexit_callback 004020a8     ucrt:api-ms-win-crt-runtime-l1-1-0.dll
 0002:000000ac       __imp___configure_narrow_argv 004020ac     ucrt:api-ms-win-crt-runtime-l1-1-0.dll
 0002:000000b0       __imp___register_onexit_function 004020b0     ucrt:api-ms-win-crt-runtime-l1-1-0.dll
 0002:000000b4       __imp___initialize_onexit_table 004020b4     ucrt:api-ms-win-crt-runtime-l1-1-0.dll
 0002:000000b8       \177api-ms-win-crt-runtime-l1-1-0_NULL_THUNK_DATA 004020b8     ucrt:api-ms-win-crt-runtime-l1-1-0.dll
 0002:000000bc       __imp____p__commode        004020bc     ucrt:api-ms-win-crt-stdio-l1-1-0.dll
 0002:000000c0       __imp___set_fmode          004020c0     ucrt:api-ms-win-crt-stdio-l1-1-0.dll
 0002:000000c4       __imp____acrt_iob_func     004020c4     ucrt:api-ms-win-crt-stdio-l1-1-0.dll
 0002:000000c8       __imp____stdio_common_vfprintf 004020c8     ucrt:api-ms-win-crt-stdio-l1-1-0.dll
 0002:000000cc       \177api-ms-win-crt-stdio-l1-1-0_NULL_THUNK_DATA 004020cc     ucrt:api-ms-win-crt-stdio-l1-1-0.dll
 0002:000000d0       __imp__JLI_CmdToArgs@4     004020d0     jli:jli.dll
 0002:000000d4       __imp__JLI_GetStdArgc@0    004020d4     jli:jli.dll
 0002:000000d8       __imp__JLI_GetStdArgs@0    004020d8     jli:jli.dll
 0002:000000dc       __imp__JLI_Launch@56       004020dc     jli:jli.dll
 0002:000000e0       __imp__JLI_MemAlloc@4      004020e0     jli:jli.dll
 0002:000000e4       __imp__JLI_InitArgProcessing@8 004020e4     jli:jli.dll
 0002:000000e8       \177jli_NULL_THUNK_DATA    004020e8     jli:jli.dll
 0002:000000ec       ___guard_check_icall_fptr  004020ec     MSVCRT:guard_support.obj
 0002:000000f0       ___xc_a                    004020f0     MSVCRT:initializers.obj
 0002:000000f8       ___xc_z                    004020f8     MSVCRT:initializers.obj
 0002:000000fc       ___xi_a                    004020fc     MSVCRT:initializers.obj
 0002:00000108       ___xi_z                    00402108     MSVCRT:initializers.obj
 0002:0000010c       ___xp_a                    0040210c     MSVCRT:initializers.obj
 0002:00000110       ___xp_z                    00402110     MSVCRT:initializers.obj
 0002:00000114       ___xt_a                    00402114     MSVCRT:initializers.obj
 0002:00000118       ___xt_z                    00402118     MSVCRT:initializers.obj
 0002:00000120       ??_C@_05CEDPJNPL@javaw@    00402120     main.obj
 0002:00000128       ??_C@_07EBOEHGIC@?9J?9ms8m@ 00402128     main.obj
 0002:00000130       ??_C@_07JMAJNDJI@openjdk@  00402130     main.obj
 0002:0000013c       ??_C@_0BF@FJHGBKOC@_JAVA_LAUNCHER_DEBUG@ 0040213c     main.obj
 0002:00000154       ??_C@_0BN@NGFJBAGH@Windows?5original?5main?5args?3?6@ 00402154     main.obj
 0002:00000174       ??_C@_0BE@OCLPFDNJ@wwwd_args?$FL?$CFd?$FN?5?$DN?5?$CFs?6@ 00402174     main.obj
 0002:00000188       ??_C@_03MDAFIFFL@0?40@     00402188     main.obj
 0002:0000018c       ??_C@_09FMBIIKIE@11?40?424?$CL8@ 0040218c     main.obj
 0002:00000210       __load_config_used         00402210     MSVCRT:loadcfg.obj
 0002:000002b0       ___safe_se_handler_table   004022b0     <linker-defined>
 0002:00000564       ___rtc_iaa                 00402564     MSVCRT:initsect.obj
 0002:00000568       ___rtc_izz                 00402568     MSVCRT:initsect.obj
 0002:0000056c       ___rtc_taa                 0040256c     MSVCRT:initsect.obj
 0002:00000570       ___rtc_tzz                 00402570     MSVCRT:initsect.obj
 0002:000005b4       __IMPORT_DESCRIPTOR_jli    004025b4     jli:jli.dll
 0002:000005c8       __IMPORT_DESCRIPTOR_KERNEL32 004025c8     kernel32:KERNEL32.dll
 0002:000005dc       __IMPORT_DESCRIPTOR_VCRUNTIME140 004025dc     vcruntime:VCRUNTIME140.dll
 0002:000005f0       __IMPORT_DESCRIPTOR_api-ms-win-crt-stdio-l1-1-0 004025f0     ucrt:api-ms-win-crt-stdio-l1-1-0.dll
 0002:00000604       __IMPORT_DESCRIPTOR_api-ms-win-crt-runtime-l1-1-0 00402604     ucrt:api-ms-win-crt-runtime-l1-1-0.dll
 0002:00000618       __IMPORT_DESCRIPTOR_api-ms-win-crt-environment-l1-1-0 00402618     ucrt:api-ms-win-crt-environment-l1-1-0.dll
 0002:0000062c       __IMPORT_DESCRIPTOR_api-ms-win-crt-math-l1-1-0 0040262c     ucrt:api-ms-win-crt-math-l1-1-0.dll
 0002:00000640       __IMPORT_DESCRIPTOR_api-ms-win-crt-locale-l1-1-0 00402640     ucrt:api-ms-win-crt-locale-l1-1-0.dll
 0002:00000654       __IMPORT_DESCRIPTOR_api-ms-win-crt-heap-l1-1-0 00402654     ucrt:api-ms-win-crt-heap-l1-1-0.dll
 0002:00000668       __NULL_IMPORT_DESCRIPTOR   00402668     jli:jli.dll
 0003:0000000c       ___scrt_native_dllmain_reason 0040300c     MSVCRT:utility.obj
 0003:00000010       ___scrt_default_matherr    00403010     MSVCRT:matherr.obj
 0003:00000020       ___isa_enabled             00403020     MSVCRT:cpu_disp.obj
 0003:00000024       ___security_cookie_complement 00403024     MSVCRT:gs_cookie.obj
 0003:00000028       ___security_cookie         00403028     MSVCRT:gs_cookie.obj
 0003:0000002c       ___scrt_ucrt_dll_is_in_use 0040302c     MSVCRT:ucrt_stubs.obj
 0003:00000030       ___scrt_current_native_startup_state 00403030     MSVCRT:utility.obj
 0003:00000034       ___scrt_native_startup_lock 00403034     MSVCRT:utility.obj
 0003:00000058       ?__type_info_root_node@@3U__type_info_node@@A 00403058     MSVCRT:tncleanup.obj
 0003:00000060       ?_OptionsStorage@?1??__local_stdio_scanf_options@@9@4_KA 00403060     MSVCRT:default_local_stdio_options.obj
 0003:00000068       ___scrt_debugger_hook_flag 00403068     MSVCRT:utility_desktop.obj
 0003:0000006c       ___isa_available           0040306c     MSVCRT:cpu_disp.obj
 0003:00000070       ___favor                   00403070     MSVCRT:cpu_disp.obj
 0003:00000398       ?_OptionsStorage@?1??__local_stdio_printf_options@@9@9 00403398     <common>
 0003:000003a0       ___initenv                 004033a0     <common>
 0003:000003a4       ___dyn_tls_dtor_callback   004033a4     <common>
 0003:000003a8       ___dyn_tls_init_callback   004033a8     <common>

 entry point at        0001:00000388

 Static symbols

 0000:ffff4000       .debug$S                   00400000     vcruntime:VCRUNTIME140.dll
 0000:ffff4000       .debug$S                   00400000     jli:jli.dll
 0000:ffff4000       .debug$S                   00400000     jli:jli.dll
 0000:ffff4000       .debug$S                   00400000     jli:jli.dll
 0000:ffff4000       .debug$S                   00400000     jli:jli.dll
 0000:ffff4000       .debug$S                   00400000     jli:jli.dll
 0000:ffff4000       .debug$S                   00400000     jli:jli.dll
 0000:ffff4000       .debug$S                   00400000     kernel32:KERNEL32.dll
 0000:ffff4000       .debug$S                   00400000     kernel32:KERNEL32.dll
 0000:ffff4000       .debug$S                   00400000     kernel32:KERNEL32.dll
 0000:ffff4000       .debug$S                   00400000     kernel32:KERNEL32.dll
 0000:ffff4000       .debug$S                   00400000     kernel32:KERNEL32.dll
 0000:ffff4000       .debug$S                   00400000     kernel32:KERNEL32.dll
 0000:ffff4000       .debug$S                   00400000     kernel32:KERNEL32.dll
 0000:ffff4000       .debug$S                   00400000     kernel32:KERNEL32.dll
 0000:ffff4000       .debug$S                   00400000     kernel32:KERNEL32.dll
 0000:ffff4000       .debug$S                   00400000     kernel32:KERNEL32.dll
 0000:ffff4000       .debug$S                   00400000     ucrt:api-ms-win-crt-runtime-l1-1-0.dll
 0000:ffff4000       .debug$S                   00400000     ucrt:api-ms-win-crt-runtime-l1-1-0.dll
 0000:ffff4000       .debug$S                   00400000     ucrt:api-ms-win-crt-runtime-l1-1-0.dll
 0000:ffff4000       .debug$S                   00400000     ucrt:api-ms-win-crt-runtime-l1-1-0.dll
 0000:ffff4000       .debug$S                   00400000     ucrt:api-ms-win-crt-runtime-l1-1-0.dll
 0000:ffff4000       .debug$S                   00400000     ucrt:api-ms-win-crt-runtime-l1-1-0.dll
 0000:ffff4000       .debug$S                   00400000     ucrt:api-ms-win-crt-runtime-l1-1-0.dll
 0000:ffff4000       .debug$S                   00400000     ucrt:api-ms-win-crt-runtime-l1-1-0.dll
 0000:ffff4000       .debug$S                   00400000     ucrt:api-ms-win-crt-stdio-l1-1-0.dll
 0000:ffff4000       .debug$S                   00400000     ucrt:api-ms-win-crt-heap-l1-1-0.dll
 0000:ffff4000       .debug$S                   00400000     ucrt:api-ms-win-crt-locale-l1-1-0.dll
 0000:ffff4000       .debug$S                   00400000     ucrt:api-ms-win-crt-runtime-l1-1-0.dll
 0000:ffff4000       .debug$S                   00400000     ucrt:api-ms-win-crt-runtime-l1-1-0.dll
 0000:ffff4000       .debug$S                   00400000     ucrt:api-ms-win-crt-runtime-l1-1-0.dll
 0000:ffff4000       .debug$S                   00400000     ucrt:api-ms-win-crt-stdio-l1-1-0.dll
 0000:ffff4000       .debug$S                   00400000     ucrt:api-ms-win-crt-runtime-l1-1-0.dll
 0000:ffff4000       .debug$S                   00400000     ucrt:api-ms-win-crt-runtime-l1-1-0.dll
 0000:ffff4000       .debug$S                   00400000     ucrt:api-ms-win-crt-runtime-l1-1-0.dll
 0000:ffff4000       .debug$S                   00400000     ucrt:api-ms-win-crt-runtime-l1-1-0.dll
 0000:ffff4000       .debug$S                   00400000     ucrt:api-ms-win-crt-runtime-l1-1-0.dll
 0000:ffff4000       .debug$S                   00400000     ucrt:api-ms-win-crt-runtime-l1-1-0.dll
 0000:ffff4000       .debug$S                   00400000     ucrt:api-ms-win-crt-runtime-l1-1-0.dll
 0000:ffff4000       .debug$S                   00400000     ucrt:api-ms-win-crt-math-l1-1-0.dll
 0000:ffff4000       .debug$S                   00400000     ucrt:api-ms-win-crt-runtime-l1-1-0.dll
 0000:ffff4000       .debug$S                   00400000     ucrt:api-ms-win-crt-runtime-l1-1-0.dll
 0000:ffff4000       .debug$S                   00400000     ucrt:api-ms-win-crt-environment-l1-1-0.dll
 0000:ffff4000       .debug$S                   00400000     ucrt:api-ms-win-crt-environment-l1-1-0.dll
 0000:ffff4000       .debug$S                   00400000     ucrt:api-ms-win-crt-runtime-l1-1-0.dll
 0000:ffff4000       .debug$S                   00400000     ucrt:api-ms-win-crt-runtime-l1-1-0.dll
 0000:ffff4000       .debug$S                   00400000     ucrt:api-ms-win-crt-stdio-l1-1-0.dll
 0000:ffff4000       .debug$S                   00400000     ucrt:api-ms-win-crt-stdio-l1-1-0.dll
 0000:ffff4000       .debug$S                   00400000     kernel32:KERNEL32.dll
 0000:ffff4000       .debug$S                   00400000     kernel32:KERNEL32.dll
 0000:ffff4000       .debug$S                   00400000     vcruntime:VCRUNTIME140.dll
 0000:ffff4000       .debug$S                   00400000     vcruntime:VCRUNTIME140.dll
 0000:ffff4000       .debug$S                   00400000     kernel32:KERNEL32.dll
 0000:ffff4000       .debug$S                   00400000     kernel32:KERNEL32.dll
 0001:00000147       ?pre_c_initialization@@YAHXZ 00401147 f   MSVCRT:exe_winmain.obj
 0001:000001f2       ?post_pgo_initialization@@YAHXZ 004011f2 f   MSVCRT:exe_winmain.obj
 0001:000001fa       ?pre_cpp_initialization@@YAXXZ 004011fa f   MSVCRT:exe_winmain.obj
 0001:0000020c       ?__scrt_common_main_seh@@YAHXZ 0040120c f   MSVCRT:exe_winmain.obj
 0001:00000392       ?find_pe_section@@YAPAU_IMAGE_SECTION_HEADER@@QAEI@Z 00401392 f   MSVCRT:utility.obj
 0001:0000060f       ___get_entropy             0040160f f   MSVCRT:gs_support.obj
 0001:00000960       $$000000                   00401960     MSVCRT:sehprolg4.obj
 0002:000000f4       ?pre_cpp_initializer@@3P6AXXZA 004020f4     MSVCRT:exe_winmain.obj
 0002:00000100       ?pre_c_initializer@@3P6AHXZA 00402100     MSVCRT:exe_winmain.obj
 0002:00000104       ?post_pgo_initializer@@3P6AHXZA 00402104     MSVCRT:exe_winmain.obj
 0002:00000138       _const_cpwildcard          00402138     main.obj
 0002:00000139       _const_disable_argfile     00402139     main.obj
 0002:00000198       _GS_ExceptionPointers      00402198     MSVCRT:gs_report.obj
 0002:00000578       __sehtable$?__scrt_common_main_seh@@YAHXZ 00402578     MSVCRT:exe_winmain.obj
 0002:00000598       __sehtable$___scrt_is_nonwritable_in_current_image 00402598     MSVCRT:utility.obj
 0002:000007e4       .idata$6                   004027e4     jli:jli.dll
 0002:0000092c       .idata$6                   0040292c     kernel32:KERNEL32.dll
 0002:0000095e       .idata$6                   0040295e     vcruntime:VCRUNTIME140.dll
 0002:00000b7a       .idata$6                   00402b7a     ucrt:api-ms-win-crt-stdio-l1-1-0.dll
 0002:00000b9a       .idata$6                   00402b9a     ucrt:api-ms-win-crt-runtime-l1-1-0.dll
 0002:00000bbc       .idata$6                   00402bbc     ucrt:api-ms-win-crt-environment-l1-1-0.dll
 0002:00000be2       .idata$6                   00402be2     ucrt:api-ms-win-crt-math-l1-1-0.dll
 0002:00000c02       .idata$6                   00402c02     ucrt:api-ms-win-crt-locale-l1-1-0.dll
 0002:00000c24       .idata$6                   00402c24     ucrt:api-ms-win-crt-heap-l1-1-0.dll
 0003:00000000       _const_progname            00403000     main.obj
 0003:00000004       _const_jargs               00403004     main.obj
 0003:00000008       _const_launcher            00403008     main.obj
 0003:00000038       ?is_initialized_as_dll@@3_NA 00403038     MSVCRT:utility.obj
 0003:00000039       ?module_local_atexit_table_initialized@@3_NA 00403039     MSVCRT:utility.obj
 0003:0000003c       ?module_local_atexit_table@@3U_onexit_table_t@@A 0040303c     MSVCRT:utility.obj
 0003:00000048       ?module_local_at_quick_exit_table@@3U_onexit_table_t@@A 00403048     MSVCRT:utility.obj
 0003:00000078       _GS_ExceptionRecord        00403078     MSVCRT:gs_report.obj
 0003:000000c8       _GS_ContextRecord          004030c8     MSVCRT:gs_report.obj
 0004:00000270       $R000000                   00404270     javaw.exe.res
 0004:00000578       $R000308                   00404578     javaw.exe.res
 0004:000006a0       $R000430                   004046a0     javaw.exe.res
 0004:00000c08       $R000998                   00404c08     javaw.exe.res
 0004:00001070       $R000E00                   00405070     javaw.exe.res
 0004:00001358       $R0010E8                   00405358     javaw.exe.res
 0004:00001c00       $R001990                   00405c00     javaw.exe.res
 0004:00002ca8       $R002A38                   00406ca8     javaw.exe.res
 0004:00003310       $R0030A0                   00407310     javaw.exe.res
 0004:000041b8       $R003F48                   004081b8     javaw.exe.res
 0004:00006760       $R0064F0                   0040a760     javaw.exe.res
